:020000000C945E
:1000020024040C9400000C9400000C9400000C9446
:1000120000000C947D040C9400000C9456040C9483
:1000220000000C9400000C9400000C9400000C944E
:1000320094170C9400000C9400000C9400000C9493
:1000420000000C9400000C9400000C9400000C942E
:1000520000000C9400000C9400000C9400000C941E
:1000620000000C9400000C9400000C9400000C940E
:1000720000000C9400000C9400000C9400000C94FE
:1000820000000C9400000C9400001027E8036400A8
:100092000A000100001000011000010020202020B1
:1000A20020CFD0CECFD3D1D2C8D2DC202020202066
:1000B20000002020202020CDC0D1D2D0CEC8D2DC5A
:1000C20020202020202000002020202020CFD0CE61
:1000D200CFD3D1D2C8D2DC20202020200000202083
:1000E200202020CDC0D1D2D0CEC8D2DC20202020EA
:1000F200202000002020202020CFD0CECFD3D1D26C
:10010200C8D2DC202020202000002020202020CD6A
:10011200C0D1D2D0CEC8D2DC2020202020200000A6
:100122002020202020CFD0CECFD3D1D2C8D2DC20E5
:100132002020202000002020202020CDC0D1D2D09D
:10014200CEC8D2DC20202020202000002020202029
:10015200202020202020202020202020202020209D
:1001620000202020CFD0CED6C5D1D120D0C0C1CE44
:10017200D2DB2020200020202020CDCEC2C0DF20D4
:10018200CFC0C9CAC0202020200020CFD0CEC4CEEC
:10019200CBC6C5CDC8C520CFC0C9CAC82020002043
:1001A2002020C4CECF2E20CDC0D1D2D0CEC9CAC835
:1001B2002020200020202020D0C5C6C8CC20D0C0BE
:1001C200C1CED2DB2020202000202020202020D1E0
:1001D200D2C0CDD6C8DF2020202020202000C2C5DA
:1001E200D0D5CDC8C920CDC0C3D0C5C2C0D2C5CB21
:1001F200DC00202020CFCEC4CEC3D0C5C220CFCBBE
:10020200C0D2DB202020002020202020D0C5C1CE5B
:10021200CBCBC8CDC320202020200020202020D0FE
:10022200D3D7CDCEC920D0C5C6C8CC20202020002F
:10023200202020CFD0CED4C8CBDC20CFC0C9CAC8A2
:1002420020202020002020202020536E36332F50E3
:100252006233372020202020200020202020202050
:100262002020536E416720202020202020200020C3
:1002720020202020CFD0CED4C8CBDC20302020209C
:10028200202020002020202020CFD0CED4C8CBDCBC
:100292002031202020202020002020202020CFD00C
:1002A200CED4C8CBDC2032202020202020002020E9
:1002B200202020CFD0CED4C8CBDC20332020202059
:1002C2002020002020202020CFD0CED4C8CBDC207C
:1002D20034202020202020002020202020CFD0CE1B
:1002E200D4C8CBDC20352020202020200020CFD0F5
:1002F200CED4C8CBDC20CFCEC4CEC3D0C5C2C020A2
:100302002000202020CFD0CED4C8CBDC20C2C5D044
:10031200D5C0202020200020CFD0CED4C8CBDC20D6
:10032200D0C5C1CECBCBC8CDC3C0200020CDC0D15B
:10033200D2D0CEC9CAC020CFD0CED4C8CBDF2020E5
:100342000020202054552B253475B0432020200056
:1003520020202020CCC5D1D2C020CFC0C9CAC820FD
:10036200202020200020202020D2C5CCCFC5D0C004
:10037200D2D3D0C0202020202000202020202020E6
:100382004B3D253275202020202020202000C2C590
:10039200D0D5CDC5C3CE20CDC0C3D0C5C2C0D2C575
:1003A200CBDF002020202020CA2DCFD0CED4C8CB36
:1003B200DF202020202020002020204D41583D25F4
:1003C200337520002020202020CCCED9CDCED1D212
:1003D200DC20202020202000CDC8C6CDC5C3CE20E1
:1003E200CDC0C3D0C5C2C0D2C5CBDF0020202050B3
:1003F2005720253475202020002020202020CCCE1C
:10040200D9CDCED1D2DC2020202020002020202ACD
:10041200C2D0C5CCDF20CFC0C9CAC82A2020202024
:10042200005425337520D1C5CA20202020542532FE
:100432007520D7C0D12000202020204D41583D25D5
:100442003375202020202020202000202020202062
:1004520020CCCED9CDCED1D2DC202020202020002D
:100462002020D2C5CCCFC5D0C0D2D3D0C020C2CAE2
:10047200CB2E20200020202020202054454D502526
:1004820033752020200020202020202020CFCBC028
:10049200D2DB202020202020202000D2C5CCCFC5B6
:1004A200D0C0D2D3D0C020CDC0C3D0C5C2C00020DE
:1004B2002020D0C5C6C8CC20CACECDD2D0CECBDF6C
:1004C2002020200020202020202AC2CACBDED7C52F
:1004D200CD2A2020202020200020202020202AC2D7
:1004E200DBCACBDED7C5CD2A20202020200020D495
:1004F200D3CDCAD6C8DF20C4CECDC0C3D0C5C2C0FA
:100502002020002020202020C4CECDC0C3D0C5C2D0
:10051200C020202020202000202020D2C5CCCF2E99
:10052200C4CECDC0C3D0C5C2C02020200020202010
:100532002020E2E5F0F1E8FF20332E3320202020B6
:100542002000202020C4CECFCECBCDC8D2C5CBDC5C
:10055200CDDBC5202020002020202020CDC0D1D2FC
:10056200D0CEC9CAC8202020202020002020202050
:100572002ACFD0CECFD3D1D2C8D2DC2A202020207D
:1005820000202AC4C0D2D7C8CA20312028C2C5D070
:10059200D5292A2020002AC4C0D2D7C8CA20322096
:1005A20028CDC8C6CDC8C9292A2000202020CFD0F6
:1005B200C5C420D3D1D2C0CDCEC2CAC8202020000B
:1005C200202020202020DFD0CACED1D2DC20202043
:1005D2002020202000202020202054552533752063
:1005E2002020202020002020202020544425337564
:1005F20020202020202000202020202020205455B0
:10060200253375202020202020202000202020209B
:1006120020D3D1D2C0CDCEC2C8D2DC20202020200F
:10062200002020CDC0D7C0D2DC20D0C0C1CED2D3D2
:1006320020CFCE202000C7C0C4C0CDCDDBCC20D37C
:10064200D1D2C0CDCEC2CAC0CC002054442533750D
:10065200B0432C20205455253375B0430020544418
:10066200253375B04300202020CDC0D7C0D2DC2076
:10067200D0C0C1CED2D320202020002020C220D042
:10068200D3D7CDCECC20D0C5C6C8CCC52020200023
:10069200543D2025750A4700533D2025750A530015
:1006A2004E3D2025750A57004B3D2025750A560000
:1006B200503D332E330A52004F3D73740A530047A4
:1006C2003D73740A5300523DD1F2E0EDF6E8FF0AA1
:1006D2005700523DC2C5D0D50A5700523DCFEEE475
:1006E200EEE3F0E5E20A5700523DD0E5E1EEEBEB36
:1006F200E8EDE30A5700523DD0F3F7EDEEE90A5771
:1007020000503D536E36332F506233370A57005034
:100712003D536E41670A5700503DCFF0EEF4E8EBCF
:10072200FC20300A5700503DCFF0EEF4E8EBFC20FD
:10073200310A5700503DCFF0EEF4E8EBFC20320ACC
:100742005700503DCFF0EEF4E8EBFC20330A57009F
:10075200503DCFF0EEF4E8EBFC20340A5700503D58
:10076200CFF0EEF4E8EBFC20350A5700503DCDE522
:10077200F20A5700D1D2C0CDD6C8DF202000C2C5B0
:10078200D0D5202020202000CFCEC4CEC3D0C5C2D9
:100792002000D0C5C1CECBCBC8CDC30020536E360E
:1007A200332F5062333700202020202020536E4107
:1007B2006700CFD0CED4C8CBDC203000CFD0CED48F
:1007C200C8CBDC203100CFD0CED4C8CBDC20320065
:1007D200CFD0CED4C8CBDC203300CFD0CED4C8CB40
:1007E200DC203400CFD0CED4C8CBDC20350048C8C2
:1007F200C7202020202A4250454DDF2A2020424592
:100802005058202000505725337520202A25347552
:100812002A202050572533750074253375B04320A4
:1008220074253375B0432074253375B0430080C0FE
:1008320001002D4E414E000002004A053008010021
:10084200510532080000F894EE27ECBBF1E0F5BF49
:10085200E5BFE0936C00F8E1F1BDE1BD8DE0A2E0FF
:10086200BB27ED938A95E9F780E090E1A0E0B1E043
:10087200ED930197E9F7EAE3F8E085919591009706
:1008820061F0A591B59105901590BF01F001059019
:100892000D920197E1F7FB01F0CFEFEFEDBFE0E141
:1008A200EEBFC0E0D5E00C94AD1A0E949C220E94DB
:1008B200AA220E94B1220E94B8220E94BF22AA2428
:1008C200BB2455240E94C622AEE1B0E00E94CD2294
:1008D2000E94D2220E94D2220E94E022E991EFBF1E
:1008E200F991E991B991A991999189917991699136
:1008F200F9901990099018950E949C220E94CF1F8E
:10090200989B49C00E94E922E3E6F1E00E94062397
:100912000E940A23999B04C00E9410230E9415235F
:10092200999902C0A895FCCF0E941A239A9B04C0F1
:100932000E9410230E9420239A9902C0A895FCCFFE
:100942000E941A230E941023E33028F0A0E0B0E0B6
:10095200E0E00E94282B0E9410230E94252329F404
:100962000E940A23E8E7F1E011C0E130A0E0FA07B3
:1009720029F40E940A23ECE8F1E008C0E230A0E08A
:10098200FA0741F40E940A23E1EAF1E0FA93EA93BA
:100992000E941B20B5CF0E9428230E941023E23020
:1009A20010F00C942705989B4FC00E94E922E6EBB9
:1009B200F1E00E940623999B03C0F30131973F01A6
:1009C200999902C0A895FCCF0E941A239A9B03C052
:1009D200F30131963F019A9902C0A895FCCF0E947B
:1009E2001A230E94302310F466247724062C072849
:1009F20031F40E940A23EBECF1E00E9406230E94EC
:100A0200352331F40E940A23E0EEF1E00E9406232E
:100A12000E943A2331F40E940A23E4EFF1E00E949B
:100A220006230E943F2331F40E940A23E9E0F2E008
:100A32000E9406230E94302331F40E940A23EDE132
:100A4200F2E00E940623AFCF0E9428230E941023C7
:100A5200E23010F00C943206062C072811F00C94A8
:100A62003206989BFCC00E94E922E2E3F2E00E9477
:100A7200062399994A94999902C0A895FCCF0E949D
:100A82001A239A9943949A9902C0A895FCCF0E947E
:100A92001A23E7E0E41508F444244420C1F40E9438
:100AA2000A230E9444230E944723A2E6B0E00E9448
:100AB20070230E947723A8E3B0E00E948023AAE378
:100AC200B0E00E9487230E948E230E949923E1E0D6
:100AD200E415C1F40E940A230E94A0230E94A323CA
:100AE200A4E6B0E00E9470230E94CC23A2E4B0E00E
:100AF2000E948023A4E4B0E00E9487230E94D523B1
:100B02000E949923E2E0E415C1F40E940A230E94A4
:100B1200E0230E94E323A6E6B0E00E9470230E9435
:100B22000C24ACE4B0E00E948023AEE4B0E00E946A
:100B320087230E9415240E949923E3E0E415D1F44F
:100B42000E940A23E6E8F2E00E9406230E94202483
:100B5200A2E7B0E00E9470230E944924A6E7B0E019
:100B62000E948023A8E7B0E00E9487230E945224BB
:100B72000E949923E4E0E415D1F40E940A23EBE9F0
:100B8200F2E00E9406230E945D24A4E8B0E00E94E5
:100B920070230E948624A8E8B0E00E948023AAE87D
:100BA200B0E00E9487230E948F240E949923E5E0EF
:100BB200E415D1F40E940A23E0EBF2E00E9406233E
:100BC2000E949A24A6E9B0E00E9470230E94C324E6
:100BD200AAE9B0E00E948023ACE9B0E00E9487233A
:100BE2000E94CC240E949923E6E0E415D1F40E94ED
:100BF2000A23E5ECF2E00E9406230E94D724A8EA29
:100C0200B0E00E9470230E940025ACEAB0E00E948E
:100C12008023AEEAB0E00E9487230E9409250E9449
:100C22009923E7E0E415D1F40E940A23EAEDF2E009
:100C32000E9406230E941425AAEBB0E00E947023B2
:100C42000E943D25AEEBB0E00E948023A0ECB0E014
:100C52000E9487230E9446250E94992302CF0E9468
:100C620051250E941023E23010F00C948C060E9451
:100C72003A2311F00C948C060E94CF1F989B47C018
:100C82000E94E922EFEEF2E00E94062399998A94EB
:100C9200999902C0A895FCCF0E941A239A9983942D
:100CA2009A9902C0A895FCCF0E941A23E2E0E815A7
:100CB20008F48824882061F40E940A230E944423B5
:100CC2000E9459250E946C25A4ECB0E00E94732575
:100CD200E1E0E81561F40E940A230E94A0230E9429
:100CE2007B250E946C25ABECB0E00E947325E2E00C
:100CF200E81561F40E940A230E94E0230E948E25D7
:100D02000E946C25A2EDB0E00E947325B7CF0E942D
:100D1200A1250E94CF1F0E941023E23010F00C94F4
:100D2200E0060E94352311F00C94E0060E94CF1FCA
:100D3200989B43C00E94E922E4E0F3E00E9406236C
:100D42009999DA94999902C0A895FCCF0E941A2326
:100D52009A99D3949A9902C0A895FCCF0E941A231B
:100D6200E2E0ED1508F4DD24DD2041F40E940A23BF
:100D72000E9444230E94A7250E94B225E1E0ED15BE
:100D820061F40E940A230E94A023ABEDB0E00E940E
:100D9200B925ADEDB0E00E94B225E2E0ED1561F4B7
:100DA2000E940A230E94E023AFEDB0E00E94B92521
:100DB200A1EEB0E00E94B225BBCF0E9451250E9455
:100DC2001023E23010F00C9468070E943F2311F0C8
:100DD2000C9468070E94CF1F989B77C00E94E9225B
:100DE200E9E1F3E00E9406239999CA94999902C015
:100DF200A895FCCF0E941A239A99C3949A9902C08B
:100E0200A895FCCF0E941A23E4E0EC1508F4CC2448
:100E1200CC2051F40E940A230E9444230E94C02540
:100E2200A9EEB0E00E94CB25E1E0EC1581F40E942E
:100E32000A230E94A023ABEDB0E00E94D225ADEEC2
:100E4200B0E00E946C25AFEEB0E00E94CB25E2E05C
:100E5200EC1581F40E940A230E94E023A3EFB0E084
:100E62000E94D225A3EFB0E00E946C25A5EFB0E06E
:100E72000E94CB25E3E0EC1591F40E940A23E6E8F8
:100E8200F2E00E940623A9EFB0E00E94D225A9EF6A
:100E9200B0E00E946C25ABEFB0E00E94CB25E4E00D
:100EA200EC1591F40E940A23EBE9F2E00E9406237A
:100EB200AFEFB0E00E94D225AFEFB0E00E946C2508
:100EC200A1E0B1E00E94CB2587CF0E9451250E946C
:100ED2001023E23010F00C94B807062C072811F00A
:100EE2000C94B807989B41C00E94E9220E94D92520
:100EF2000E940A230E94DC25999B04C00E94E225DD
:100F02000E94E725999902C0A895FCCF0E941A2356
:100F12009A9B04C00E94E2250E94EC259A9902C085
:100F2200A895FCCF0E941A230E94E225329720F056
:100F3200A6E0B0E00E94CD220E94E225309741F463
:100F42000E94F125EEE9F0E00E94CA2C0E94F625EB
:100F52000E94E225319741F40E94F125E4EBF0E092
:100F62000E94CA2C0E94F625BDCF0E9428230E940F
:100F72001023E23010F00C9409080E943A2311F079
:100F82000C940908989B42C00E94E9220E94D9252C
:100F92000E940A230E94DC25999B04C00E94FD2521
:100FA2000E941523999902C0A895FCCF0E941A238A
:100FB2009A9B04C00E94FD250E9420239A9902C098
:100FC200A895FCCF0E941A230E94FD25E23028F04A
:100FD200A1E0B0E0E0E00E94282B0E94FD25E03075
:100FE20041F40E94F125EAECF0E00E94CA2C0E9432
:100FF200F6250E94FD25E13041F40E94F125E0EE44
:10100200F0E00E94CA2C0E94F625BCCF0E94282341
:101012000E941023E23010F00C945A080E943523EB
:1010220011F00C945A08989B42C00E94E9220E9437
:10103200D9250E940A230E94DC25999B04C00E94A4
:1010420002260E941523999902C0A895FCCF0E94FE
:101052001A239A9B04C00E9402260E9420239A9976
:1010620002C0A895FCCF0E941A230E940226E230F9
:1010720028F0A2E0B0E0E0E00E94282B0E940226C5
:10108200E03041F40E94F125E6EFF0E00E94CA2C24
:101092000E94F6250E940226E13041F40E94F125C9
:1010A200ECE0F1E00E94CA2C0E94F625BCCF0E941F
:1010B20028230E941023E23010F00C94AB080E9407
:1010C2003F2311F00C94AB08989B42C00E94E92286
:1010D2000E94D9250E940A230E94DC25999B04C004
:1010E2000E9407260E941523999902C0A895FCCF59
:1010F2000E941A239A9B04C00E9407260E94202362
:101102009A9902C0A895FCCF0E941A230E94072632
:10111200E23028F0A3E0B0E0E0E00E94282B0E9439
:101122000726E03041F40E94F125E2E2F1E00E945C
:10113200CA2C0E94F6250E940726E13041F40E9443
:10114200F125E8E3F1E00E94CA2C0E94F625BCCF0B
:101152000E9428230E941023E23010F00C942B09E5
:10116200062C072811F00C942B09989B67C00E944B
:101172000A230E940C260E940F260E9414260E9417
:101182002B260E943626999B04C00E943E260E946E
:1011920043269A9B04C00E943E260E944C260E942F
:1011A200552610F00E94AA22E42D0E94252329F43C
:1011B2000E945D26A2E3B0E03EC0E130A0E0FA0763
:1011C20029F40E945D26ACE3B0E035C0E230A0E035
:1011D200FA0729F40E945D26A6E4B0E02CC0E330B1
:1011E200A0E0FA0729F40E945D26A8E6B0E023C039
:1011F200E430A0E0FA0729F40E945D26AAE7B0E0F5
:101202001AC0E530A0E0FA0729F40E945D26ACE896
:10121200B0E011C0E630A0E0FA0729F40E945D2692
:10122200AEE9B0E008C0E730A0E0FA0731F40E946E
:101232005D26A0EBB0E00E94202B97CF0E943A23BC
:1012420011F40E94BF220E943A2311F40E94AA22A2
:101252000E9428230E941023E23010F00C947E0991
:101262000E94352311F00C947E09989B3AC00E948B
:101272000A230E940C260E940F260E9414260E9416
:101282002B260E943626999B04C00E943E260E946D
:1012920043269A9B04C00E943E260E944C260E942E
:1012A200552610F00E94AA22ED2D0E94252329F432
:1012B2000E945D26A7EDB0E011C0E130A0E0FA0780
:1012C20029F40E945D26ABEDB0E008C0E230A0E058
:1012D200FA0731F40E945D26AFEDB0E00E94202BA8
:1012E200C4CF0E943A2311F40E94BF220E943A23E3
:1012F20011F40E94AA220E9428230E941023E230A5
:10130200B0F50E94302399F5989B2FC00E940A23C2
:101312000E940C260E940F260E9462260E946726C7
:101322000E946C260E942B260E943626999B06C09C
:101332000E9467260E94E7250E947B269A9B06C090
:101342000E9467260E94EC250E947B260E94672647
:10135200ED32A1E0FA0720F0A3E0B1E00E94CD2235
:10136200A3E0B1E00E94B925CFCF0E9428230E94BA
:101372001023E23010F00C94410A062C072811F0D9
:101382000C94410A0E94E225319711F00C94410A13
:10139200989B74C00E940A230E940C260E940F266A
:1013A2000E9481260E948A260E9495260E949A26E1
:1013B200999B06C00E949D260E94E7250E947B26DB
:1013C2009A9B06C00E949D260E94EC250E947B26C5
:1013D2000E949D26B49710F00E94A2260E949D268C
:1013E2003F9710F40E94A226E42D0E94252329F49F
:1013F2000E949D26A6E5B0E03EC0E130A0E0FA07DB
:1014020029F40E949D26A8E5B0E035C0E230A0E0B4
:10141200FA0729F40E949D26AAE5B0E02CC0E33029
:10142200A0E0FA0729F40E949D26AEE6B0E023C0B0
:10143200E430A0E0FA0729F40E949D26A0E8B0E07B
:101442001AC0E530A0E0FA0729F40E949D26A2E91D
:10145200B0E011C0E630A0E0FA0729F40E949D2610
:10146200A4EAB0E008C0E730A0E0FA0731F40E9435
:101472009D26A6EBB0E00E94202B8ACF0E94282353
:101482000E941023E23010F00C94D60A062C072892
:1014920011F00C94D60A0E94E225319711F00C94B7
:1014A200D60A989B80C00E940A230E940C260E94A2
:1014B2000F26EAEBF3E0FA93EA930E94A9260E9430
:1014C200AE260E948A260E949526E6ECF3E00E9450
:1014D2000623999B04C0A7E3B5E00E94BD269A9B10
:1014E20004C0A7E3B5E00E94C026A0913705B091E1
:1014F2003805A436E0E0BE0714F00E94C326A0918E
:101502003805AA2332F4E0E0F0E0E0933705F093E7
:101512003805E42D0E94252329F40E94A926A5E07E
:10152200B1E03EC0E130A0E0FA0729F40E94A9260A
:10153200A7E0B1E035C0E230A0E0FA0729F40E944A
:10154200A926A9E0B1E02CC0E330A0E0FA0729F413
:101552000E94A926ABE0B1E023C0E430A0E0FA0784
:1015620029F40E94A926ADE0B1E01AC0E530A0E05E
:10157200FA0729F40E94A926AFE0B1E011C0E630D3
:10158200A0E0FA0729F40E94A926A1E1B1E008C06F
:10159200E730A0E0FA0731F40E94A926A3E1B1E006
:1015A2000E94202B7ECF0E9428230E941023E2302B
:1015B20010F00C94320B0E94352311F00C94320B74
:1015C2000E940226E13011F00C94320B989B47C026
:1015D2000E940A230E940C260E940F260E94812646
:1015E2000E948A260E9495260E949A26999B06C0EE
:1015F2000E949D260E94E7250E947B269A9B06C098
:101602000E949D260E94EC250E947B260E949D2618
:10161200B49710F00E94A2260E949D263F9710F4D4
:101622000E94A226ED2D0E94252329F40E949D26C8
:10163200A9EDB0E011C0E130A0E0FA0729F40E9460
:101642009D26ADEDB0E008C0E230A0E0FA0731F42B
:101652000E949D26A1EEB0E00E94202BB7CF0E94EF
:1016620028230E941023E23010F00C94B80B062CB1
:10167200072811F00C94B80B0E94E225319711F063
:101682000C94B80B989B67C00E940A230E940C26F8
:101692000E940F260E9462260E94CA260E946C2681
:1016A2000E94CF260E943626999B02C00E94DA260B
:1016B2009A9B02C00E94DD260E94E02610F00E9442
:1016C200B122E42D0E94252329F40E94CA26A4E314
:1016D200B0E03EC0E130A0E0FA0729F40E94CA2639
:1016E200AEE3B0E035C0E230A0E0FA0729F40E9490
:1016F200CA26A8E4B0E02CC0E330A0E0FA0729F43F
:101702000E94CA26AAE6B0E023C0E430A0E0FA07AD
:1017120029F40E94CA26ACE7B0E01AC0E530A0E086
:10172200FA0729F40E94CA26AEE8B0E011C0E630FA
:10173200A0E0FA0729F40E94CA26A0EAB0E008C095
:10174200E730A0E0FA0731F40E94CA26A2EBB0E02B
:101752000E94202B97CF0E94352311F40E94B822B9
:101762000E94352311F40E94B1220E9428230E9474
:101772001023E23010F00C94110C0E943A2311F065
:101782000C94110C0E94FD25E13011F00C94110C07
:10179200989B3AC00E940A230E940C260E940F26A0
:1017A2000E9462260E94CA260E946C260E94CF26B0
:1017B2000E943626999B02C00E94DA269A9B02C09A
:1017C2000E94DD260E94E02610F00E94B122E82D40
:1017D2000E94252329F40E94CA26A2ECB0E011C07F
:1017E200E130A0E0FA0729F40E94CA26A9ECB0E091
:1017F20008C0E230A0E0FA0731F40E94CA26A0ED48
:10180200B0E00E94202BC4CF0E94352311F40E9425
:10181200B8220E94352311F40E94B1220E9428238B
:101822000E941023E23010F00C94750C0E943F23AA
:1018320011F00C94750C0E940726E13011F00C9403
:10184200750C989B4FC00E940A230E940C260E948E
:101852000F260E9462260E94CA260E946C260E94BF
:10186200CF260E943626999B02C00E94DA269A9BB6
:1018720002C00E94DD260E94E826A732E2E0BE07EF
:1018820010F00E94B122EC2D0E94252329F40E941F
:10189200CA26A5EEB0E023C0E130A0E0FA0729F4A1
:1018A2000E94CA26ABEEB0E01AC0E230A0E0FA070E
:1018B20029F40E94CA26A1EFB0E011C0E330A0E0F3
:1018C200FA0729F40E94CA26A7EFB0E008C0E43064
:1018D200A0E0FA0731F40E94CA26ADEFB0E00E9400
:1018E200202BAFCF0E9428230E941023E23010F059
:1018F2000C94F30C0E943F2311F00C94F30C0E9401
:101902000726E13011F00C94F30C989B69C00E94F9
:101912000A230E940C260E940F26EEEEF3E0FA93B1
:10192200EA930E94ED260E94AE260E948A260E9419
:101932009526EBEFF3E00E940623999B06C00E94D6
:10194200ED260E94E7250E947B269A9B06C00E94F4
:10195200ED260E94EC250E947B260E94ED26E536AC
:10196200A0E0FA0724F0A3EEB0E00E94F226A4EE73
:10197200B0E00E940C2BEE2322F4A3EEB0E00E9412
:10198200CD22EC2D0E94252329F40E94ED26A9EEFA
:10199200B0E023C0E130A0E0FA0729F40E94ED266E
:1019A200AFEEB0E01AC0E230A0E0FA0729F40E94DC
:1019B200ED26A5EFB0E011C0E330A0E0FA0729F46C
:1019C2000E94ED26ABEFB0E008C0E430A0E0FA07D9
:1019D20031F40E94ED26A1E0B1E00E94202B95CFC8
:1019E2000E9428230E941023E23010F00C94AD0DC7
:1019F2000E943F2311F00C94AD0D0E940726E130A6
:101A020011F00C94AB0D989BA5C00E94F7260E9482
:101A12000C260E94FD260E940C260E949526EEE0CE
:101A2200F4E00E9406230E940F26E3E2F4E0FA9318
:101A3200EA93E0911F05F09120050E940327E091AF
:101A42001D05F0911E050E9403270E9408270E948F
:101A52000A230E940F260E940E20999B1AC00E9400
:101A62007B260E940D273197604070400E94182B00
:101A7200EF5FFF4F6F4F7F4FAFE1B5E00E9412273C
:101A82000E94182730F40E942027E0931F05F0934C
:101A920020059A9B11C00E947B260E940D27EF5FB2
:101AA200FF4F6F4F7F4F0E94182B3197604070405D
:101AB200AFE1B5E00E942927A0911F05B091200552
:101AC200A43FE1E0BE0760F0A6E1B0E0E4EFF1E0A0
:101AD20060E070E00E94182BE0931F05F093200550
:101AE2009B9B13C00E947B260E940D27E051FE4063
:101AF200604070400E942F270E9412270E941827E0
:101B020020F40E9420270E943627CF9B22C00E94E9
:101B12007B260E940D27E05FF14F6F4F7F4F0E949F
:101B22002F270E9429270E940D27E038A1E5FA07F6
:101B3200A1E06A07A0E07A0760F0A6E1B0E0E0E881
:101B4200F1E561E070E00E94182BE8E1F0E00E940C
:101B5200362759CF0E9428230E941023E23010F02A
:101B62000C94360E062C072811F00C94360E0E94A7
:101B7200E225319711F00C94360E989B74C00E94A6
:101B82000A230E940C260E940F260E943B270E94D5
:101B9200CF260E9495260E949A26999B06C00E94F3
:101BA20044270E94E7250E9449279A9B06C00E946B
:101BB20044270E94EC250E9449270E944427B4979B
:101BC20010F00E944F270E9444273F9710F40E9472
:101BD2004F27E42D0E94252329F40E944427ACE5D7
:101BE200B0E03EC0E130A0E0FA0729F40E944427A9
:101BF200AEE5B0E035C0E230A0E0FA0729F40E9479
:101C02004427A0E6B0E02CC0E330A0E0FA0729F4B4
:101C12000E944427A0E7B0E023C0E430A0E0FA0726
:101C220029F40E944427A2E8B0E01AC0E530A0E0FF
:101C3200FA0729F40E944427A4E9B0E011C0E63073
:101C4200A0E0FA0729F40E944427A6EAB0E008C0FF
:101C5200E730A0E0FA0731F40E944427A8EBB0E095
:101C62000E94202B8ACF0E9428230E941023E23058
:101C720010F00C94CB0E062C072811F00C94CB0E0E
:101C82000E94E225319711F00C94CB0E989B80C0F4
:101C92000E940A230E940C260E940F26E9E3F4E028
:101CA200FA93EA930E9456270E94AE260E94CF26FC
:101CB2000E949526EDE4F4E00E940623999B04C05D
:101CC200A9E3B5E00E94BD269A9B04C0A9E3B5E052
:101CD2000E94C026A0913905B0913A05A436E0E0F1
:101CE200BE0714F00E945B27A0913A05AA2332F4A2
:101CF200E0E0F0E0E0933905F0933A05E42D0E942C
:101D0200252329F40E945627A5E1B1E03EC0E13027
:101D1200A0E0FA0729F40E945627A7E1B1E035C0F6
:101D2200E230A0E0FA0729F40E945627A9E1B1E0C7
:101D32002CC0E330A0E0FA0729F40E945627ABE159
:101D4200B1E023C0E430A0E0FA0729F40E9456274C
:101D5200ADE1B1E01AC0E530A0E0FA0729F40E9433
:101D62005627AFE1B1E011C0E630A0E0FA0729F44E
:101D72000E945627A1E2B1E008C0E730A0E0FA07CE
:101D820031F40E945627A3E2B1E00E94202B7ECFBD
:101D92000E9428230E941023E23010F00C94270F97
:101DA2000E943A2311F00C94270F0E94FD25E13086
:101DB20011F00C94270F989B47C00E940A230E949F
:101DC2000C260E940F260E943B270E94CF260E94CB
:101DD20095260E949A26999B06C00E9444270E943B
:101DE200E7250E9449279A9B06C00E9444270E9429
:101DF200EC250E9449270E944427B49710F00E94C4
:101E02004F270E9444273F9710F40E944F27E82D46
:101E12000E94252329F40E944427A7ECB0E011C0B8
:101E2200E130A0E0FA0729F40E944427AEECB0E0CA
:101E320008C0E230A0E0FA0731F40E944427A5ED81
:101E4200B0E00E94202BB7CF0E9428230E941023CB
:101E5200E23010F00C949C0F0E943F2311F00C947E
:101E62009C0F0E940726E13011F00C949C0F0E94F7
:101E7200E8260E94B32C10F00C949C0F989B59C03A
:101E82000E940A230E940C260E940F260E943B27D2
:101E92000E94CF260E9495260E949A26999B06C0F0
:101EA2000E9444270E94E7250E9449279A9B06C068
:101EB2000E9444270E94EC250E9449270E94442741
:101EC200B49710F00E944F270E9444273F9710F4C6
:101ED2000E944F27EC2D0E94252329F40E944427BB
:101EE200A7EEB0E023C0E130A0E0FA0729F40E9497
:101EF2004427ADEEB0E01AC0E230A0E0FA0729F4C0
:101F02000E944427A3EFB0E011C0E330A0E0FA073B
:101F120029F40E944427A9EFB0E008C0E430A0E011
:101F2200FA0731F40E944427AFEFB0E00E94202B61
:101F3200A5CF0E9428230E941023E23010F00C94B7
:101F42002F10062C072811F00C942F100E94E22566
:101F5200319711F00C942F10989B7EC00E940A2397
:101F62000E940C260E94F726E0E9F3E00E94062375
:101F72000E949526E2E6F4E00E9406230E940F26C4
:101F82000E9462270E946B270E940F260E940E2049
:101F9200999B06C00E9470270E94E7250E947B261B
:101FA2009A9B06C00E9470270E94EC250E947B2605
:101FB2000E947027EB3FA0E0FA0720F0AEE2B0E00B
:101FC2000E94CD22E42D0E94252329F40E9470272D
:101FD200A0E5B0E03EC0E130A0E0FA0729F40E949B
:101FE2007027A2E5B0E035C0E230A0E0FA0729F49C
:101FF2000E947027A4E5B0E02CC0E330A0E0FA070D
:1020020029F40E947027ACE6B0E023C0E430A0E0DF
:10201200FA0729F40E947027AEE7B0E01AC0E53053
:10202200A0E0FA0729F40E947027A0E9B0E011C0ED
:10203200E630A0E0FA0729F40E947027A2EAB0E095
:1020420008C0E730A0E0FA0731F40E947027A4EB41
:10205200B0E00E94202B80CF0E9428230E941023F0
:10206200E23010F00C9495100E943A2311F00C9477
:1020720095100E94FD25E13011F00C949510989B6B
:1020820051C00E940A230E940C260E94F726E8E80B
:10209200F4E00E9406230E949526EDE9F4E00E94F6
:1020A20006230E940F260E9462270E946B270E942D
:1020B2000F260E940E20999B06C00E9470270E9444
:1020C200E7250E947B269A9B06C00E9470270E94E9
:1020D200EC250E947B260E947027EB3FA0E0FA07C6
:1020E20020F0AEE2B0E00E94CD22E82D0E9425232E
:1020F20029F40E947027A5ECB0E011C0E130A0E005
:10210200FA0729F40E947027ACECB0E008C0E23074
:10211200A0E0FA0731F40E947027A3EDB0E00E941C
:10212200202BADCF0E9428230E941023E23010F012
:102132000C943011062C072811F00C9430110E94D7
:10214200E225319711F00C943011989B86C00E94C1
:10215200FD260E940C260E94F7260E9475270E94E7
:102162009526E1EBF4E00E940623999B04C00E94AD
:1021720078270E94E725999902C0A895FCCF0E9472
:102182001A239A9B04C00E9478270E94EC259A99F0
:1021920002C0A895FCCF0E941A230E94782732978A
:1021A20010F00E947D270E947827309721F40E9428
:1021B2000A230E9480270E947827319721F40E94E7
:1021C2000A230E948327E42D0E94252329F40E94DA
:1021D2007827A2E6B0E03EC0E130A0E0FA0729F499
:1021E2000E947827A4E6B0E035C0E230A0E0FA070A
:1021F20029F40E947827A6E6B0E02CC0E330A0E0E4
:10220200FA0729F40E947827A2E7B0E023C0E4305D
:10221200A0E0FA0729F40E947827A4E8B0E01AC0E7
:10222200E530A0E0FA0729F40E947827A6E9B0E099
:1022320011C0E630A0E0FA0729F40E947827A8EA44
:10224200B0E008C0E730A0E0FA0731F40E94782736
:10225200AAEBB0E00E94202B78CF0E9428230E9494
:102262001023E23010F00C949E110E943A2311F0D8
:102272000C949E110E94FD25E13011F00C949E11E8
:10228200989B59C00E94FD260E940C260E94F726A8
:102292000E9475270E949526E1EBF4E00E94062336
:1022A200999B04C00E9478270E94E725999902C051
:1022B200A895FCCF0E941A239A9B04C00E947827FB
:1022C2000E94EC259A9902C0A895FCCF0E941A237D
:1022D2000E947827329710F00E947D270E9478276B
:1022E200309721F40E940A230E9480270E947827B7
:1022F200319721F40E940A230E948327E82D0E942D
:10230200252329F40E948627A4ECB0E011C0E13015
:10231200A0E0FA0729F40E948627ABECB0E008C0DF
:10232200E230A0E0FA0731F40E948627A2EDB0E085
:102332000E94282BA5CF0E9428230E941023E2305E
:1023420010F00C943D12062C072811F00C943D124B
:102352000E94E225319711F00C943D12989B8AC09D
:102362000E94FD260E940C260E94F7260E947527D5
:102372000E949526E0EFF4E00E940623999B04C098
:102382000E948B270E94E725999902C0A895FCCF4D
:102392000E941A239A9B04C00E948B270E94EC255C
:1023A2009A9902C0A895FCCF0E941A230E948B27FB
:1023B200329720F0A8E0B0E00E94CD220E948B2745
:1023C200309721F40E940A230E9480270E948B27C3
:1023D200319721F40E940A230E948327E42D0E9450
:1023E200252329F40E948B27A6E3B0E03EC0E1300A
:1023F200A0E0FA0729F40E948B27A0E4B0E035C0E0
:10240200E230A0E0FA0729F40E948B27AAE4B0E0A8
:102412002CC0E330A0E0FA0729F40E948B27A4E73E
:10242200B0E023C0E430A0E0FA0729F40E948B2731
:10243200A6E8B0E01AC0E530A0E0FA0729F40E944D
:102442008B27A8E9B0E011C0E630A0E0FA0729F432
:102452000E948B27AAEAB0E008C0E730A0E0FA07A2
:1024620041F40E948B27ACEBB0E00E94202B0E942B
:10247200902774CF0E9428230E941023E23010F08C
:102482000C94DE12062C072811F00C94DE120E9426
:10249200E225319711F00C94DE120E948B273097BF
:1024A20011F00C94DC12989B86C00E940A230E94B1
:1024B2000C260E94CF1F0E94F726E5E0F5E00E945D
:1024C20006230E949526E2E6F4E00E9406230E947B
:1024D2000F26E7E7F4E0FA93EA930E9497270E9417
:1024E20003270E946B270E940F260E940E20999BB1
:1024F20006C00E9497270E94E7250E947B269A9B8E
:1025020006C00E9497270E94EC250E947B260E940B
:102512009727EB3FA0E0FA0720F0AAE0B0E00E9484
:10252200CD22E42D0E94252329F40E949727A8E3B7
:10253200B0E03EC0E130A0E0FA0729F40E949727FC
:10254200A2E4B0E035C0E230A0E0FA0729F40E942C
:102552009727ACE4B0E02CC0E330A0E0FA0729F4FE
:102562000E949727A6E7B0E023C0E430A0E0FA0774
:1025720029F40E949727A8E8B0E01AC0E530A0E04D
:10258200FA0729F40E949727AAE9B0E011C0E630C1
:10259200A0E0FA0729F40E949727ACEAB0E008C04D
:1025A200E730A0E0FA0731F40E949727AEEBB0E0E3
:1025B2000E94202B78CF0E9428230E941023E23011
:1025C20010F00C947D13062C072811F00C947D1347
:1025D2000E94E225319711F00C947D130E948B2703
:1025E200309711F00C947D13989B7AC00E94CF1FF4
:1025F2000E940A230E940C260E940F260E94622635
:102602000E949C270E946C260E94CF260E9495263B
:10261200EAE1F5E00E940623999B06C00E949C27EE
:102622000E94E7250E947B269A9B06C00E949C2757
:102632000E94EC250E947B260E949C27EB3EA1E093
:10264200FA0720F0ACE0B0E00E94CD22E42D0E9417
:10265200252329F40E949C27AAE3B0E03EC0E13082
:10266200A0E0FA0729F40E949C27A4E4B0E035C058
:10267200E230A0E0FA0729F40E949C27AEE4B0E021
:102682002CC0E330A0E0FA0729F40E949C27A8E7B7
:10269200B0E023C0E430A0E0FA0729F40E949C27AE
:1026A200AAE8B0E01AC0E530A0E0FA0729F40E94D7
:1026B2009C27ACE9B0E011C0E630A0E0FA0729F4AB
:1026C2000E949C27AEEAB0E008C0E730A0E0FA071B
:1026D20031F40E949C27A0ECB0E00E94202B84CF12
:1026E2000E94352311F40E94B8220E94352311F46E
:1026F2000E94B1220E9428230E941023E23011F08E
:102702000C94B415989B5CC00E940A23EFE2F5E09A
:102712000E9406230E949526E4E4F5E00E94062327
:102722000E94F726E9E5F5E00E94062399999A941A
:10273200999902C0A895FCCF0E941A239A99939462
:102742009A9902C0A895FCCF0E941A23E5E0E915E8
:1027520008F49924992031F40E94FD26EEE6F5E072
:102762000E940623E1E0E91531F40E94FD26E3E828
:10277200F5E00E940623E2E0E91531F40E94FD260D
:10278200E8E9F5E00E940623E3E0E91531F40E944E
:10279200FD26EEE0F4E00E940623E4E0E91531F4C0
:1027A2000E94FD26EDEAF5E00E940623E5E0E91528
:1027B20031F40E94FD26E2ECF5E00E940623A2CF4E
:1027C2000E94A125E1E0E91559F5989B29C00E94D4
:1027D2000F26E7EDF5E0FA93EA930E94A1270E9403
:1027E20003270E94A6270E940F260E940E20999B73
:1027F20006C00E94A1270E94E7250E9449279A9BB2
:1028020006C00E94A1270E94EC250E9449270E942F
:10281200A127F39720F0AAE2B0E00E94CD22D5CF03
:102822000E944927E2E0E91559F5989B29C00E94C8
:102832000F26E8EEF5E0FA93EA930E94AB270E9496
:1028420003270E94A6270E940F260E940E20999B12
:1028520006C00E94AB270E94E7250E9449279A9B47
:1028620006C00E94AB270E94EC250E9449270E94C5
:10287200AB27F39720F0ACE2B0E00E94CD22D5CF97
:10288200E3E0E91559F5989B29C00E940F26E9EF6C
:10289200F5E0FA93EA930E94B0270E9403270E9470
:1028A200A6270E940F260E940E20999B06C00E9416
:1028B200B0270E94E7250E9449279A9B06C00E94E2
:1028C200B0270E94EC250E9449270E94B027FD975D
:1028D20020F0A4E1B0E00E94CD22D5CFE4E0E915DA
:1028E20011F00C948215989B0CC10E940A23EEE011
:1028F200F6E00E940623A2E3B0E0E3ECF0E00E94DF
:10290200202BA4E3B0E00E94B527A6E3B0E00E942A
:10291200BA27ACE3B0E0E6EEF0E00E94202BAEE393
:10292200B0E00E94B527A0E4B0E00E94BA27A6E476
:10293200B0E0E6EEF0E00E94202BA8E4B0E00E94B6
:10294200B527A0E5B0E0EEE6F0E00E94202BA2E57C
:10295200B0E0E3E7F0E00E94202BA4E5B0E0E9E676
:10296200F0E00E94202BA6E5B0E00E94BF27A8E578
:10297200B0E00E94BF27AAE5B0E00E94BF27ACE505
:10298200B0E00E94BF27AEE5B0E00E94BF27A0E6FC
:10299200B0E00E94BF27A2E6B0E00E94CD22A4E6EA
:1029A200B0E00E94CD22A6E6B0E00E94CD22AAE4C9
:1029B200B0E00E94CD22ACE4B0E0E2EDF0E00E9493
:1029C200202BAEE4B0E00E94C427A4E5B0E00E9450
:1029D200F226A6E6B0E00E94CD22A2ECB0E0E0E949
:1029E200F1E00E94202BA4ECB0E0E0E00E94282B52
:1029F200A5ECB0E0E2E8F0E00E94202BA7ECB0E00A
:102A0200E8E1F0E00E94202BA5EEB0E00E94B5279D
:102A1200A7EEB0E0E8E1F0E00E94202BA9EEB0E0E2
:102A2200E0E5F0E00E94202BA0E2B0E0E0EFF0E071
:102A32000E94202BE0E0F0E00E943627A6E1B0E001
:102A4200E0E0F0E060E070E00E94182BA7EDB0E05B
:102A5200ECEDF0E00E94202BA9EDB0E0E4E1F0E023
:102A62000E94202BAAE2B0E00E94C427ACE2B0E0B0
:102A72000E94C427A4E1B0E0EAE0F0E00E94202B2B
:102A820055240E947D27A0E0B0E0E0E00E94282BC0
:102A9200662477240E94C9270E94D0270E94C6225A
:102AA2000E94D527A8E0B0E00E94BA27A2E2B0E0D7
:102AB2000E94CD22A4E2B0E00E94CD22A6E2B0E0C4
:102AC2000E94CD22A8E2B0E00E94CD22A3E0B1E0B4
:102AD200E4EBF0E00E94202B0E945B270E94C326B9
:102AE200A5E1B1E00E94F226A5E0B1E00E94F22643
:102AF200A7E1B1E00E94F226A7E0B1E00E94F2262F
:102B0200F2CEE5E0E91559F5989B29C00E940F26FF
:102B1200E9EFF5E0FA93EA930E94E0270E94032787
:102B22000E94A6270E940F260E940E20999B06C093
:102B32000E94E0270E94E7250E9449279A9B06C02F
:102B42000E94E0270E94EC250E9449270E94E0276C
:102B5200FD9720F0A7E2B1E00E94CD22D5CF0E94DE
:102B6200CF1F0E94A125062C072811F00C943C16B9
:102B7200A895989B80C00E940A230E940C260E945E
:102B820095260E94E5270E94F7260E94E8270E94C8
:102B92000F260E94EB270E94F1270E9408270E941D
:102BA200FD260E940F260E94F3270E94D5270E942D
:102BB2009027E2E3E0931005A895E42D0E942523D7
:102BC20039F40E9447230E9477230E948E234CC02F
:102BD200E130A0E0FA0739F40E94A3230E94CC233B
:102BE2000E94D52341C0E230A0E0FA0739F40E94E6
:102BF200E3230E940C240E94152436C0E330A0E097
:102C0200FA0739F40E9420240E9449240E94522487
:102C12002BC0E430A0E0FA0739F40E945D240E9440
:102C220086240E948F2420C0E530A0E0FA0739F400
:102C32000E949A240E94C3240E94CC2415C0E6302C
:102C4200A0E0FA0739F40E94D7240E9400250E94CE
:102C520009250AC0E730A0E0FA0761F40E941425B2
:102C62000E943D250E9446250E94082BE0933705CD
:102C7200F09338057ECF0E94352311F00C947E1616
:102C8200A895989B3AC0A8950E940A230E940C26F8
:102C92000E9495260E94E5270E94F7260E94E827B7
:102CA2000E940F260E94FA270E946B270E940F267D
:102CB2000E94F3270E94D5270E9490270E94B122EA
:102CC200ED2D0E94252319F40E94A7250EC0E130A4
:102CD200A0E0FA0721F0E230A0E0FA0761F4ABEDE0
:102CE200B0E00E94B925ADEDB0E00E94082BA0E152
:102CF200B0E00E94202BA895C4CF0E943A2311F085
:102D02000C94C516A895989B3FC0A8950E940A23CB
:102D12000E940C260E9495260E94E5270E94F72613
:102D22000E94E8270E940F260E94EB270E9470272C
:102D32000E9403270E9408270E94FD260E940F2658
:102D42000E94F3270E94D5270E9490270E94AA2260
:102D5200E82D0E94252319F40E9459250DC0E13067
:102D6200A0E0FA0719F40E947B2506C0E230A0E039
:102D7200FA0741F40E948E250E94082BAEE0B0E0D3
:102D82000E94202BA895BFCF0E943F2311F00C94E4
:102D92003E17A895989B71C0A8950E940A230E948D
:102DA2000C260E9495260E94E5270E94F7260E9483
:102DB200E8270E940F26EFE5F6E0FA93EA930E94D5
:102DC200CA260E9403270E946B270E940F260E9498
:102DD200F327A0E2B0E00E94CD220E94D5270E94F4
:102DE2009027A895EC2D0E94252329F40E94C02546
:102DF200A9EEB0E03BC0E130A0E0FA0759F4ABEE37
:102E0200B0E00E94D225ADEEB0E00E946C25AFEE9C
:102E1200B0E02CC0E230A0E0FA0759F4A1EFB0E034
:102E22000E94D225A3EFB0E00E946C25A5EFB0E08E
:102E32001DC0E330A0E0FA0759F4A7EFB0E00E940A
:102E4200D225A9EFB0E00E946C25ABEFB0E00EC036
:102E5200E430A0E0FA0781F4ADEFB0E00E94D225A1
:102E6200AFEFB0E00E946C25A1E0B1E00E94082B18
:102E7200A3EEB0E00E94202B8DCF0E94302321F5DB
:102E8200A895989B21C0A8950E940A230E940C260F
:102E92000E949526E8E6F6E00E9406230E94F726A5
:102EA200EDE7F6E00E9406230E940F260E94FA2711
:102EB2000E946B270E940F260E94F3270E94D527AB
:102EC2000E949027A895DDCF0E941023E030E1F404
:102ED200A5E2B1E00E94CD220E94FF270E940228B3
:102EE200AA24BB240E94C927E0931305F09314057A
:102EF2000E94C622E0E0F0E00E94D027E0E0F0E08D
:102F0200E0931505F09316050E941023E23041F478
:102F1200A8E0B0E00E94BA270E94B1220E94AA2231
:102F22000E94CF1F9DC10E949C220E9405280E94E0
:102F3200CA26EA1BFB0BE0932D05F0932E05062C07
:102F42000728B1F40E940A282CF00E94112812F4DA
:102F52000E94B8220E940A285CF4A0913605AA2396
:102F620012F40E94B8220E941E2814F00E94262801
:102F72000E94352311F40E94B8220E943A23E1F400
:102F82000E940A282CF00E94112812F40E94B822F2
:102F92000E940A288CF4A0913605AA2312F40E94FA
:102FA200B8220E941E2814F00E9426280E942D2872
:102FB200E0932705F09328050E943F2349F40E94DD
:102FC200E826129728F00E94322810F00E94372833
:102FD200A0912505B09126050E943C28EA1BFB0B17
:102FE200E0932F05F09330050E9441280E945D2650
:102FF200EA1BFB0BE0933105F0933205E1E0E515A6
:10300200E1F4062C0728C9F40E9446280E94B32C3A
:1030120054F40E944628159734F40E944B280E94CB
:1030220050280E9455280E946B283CF40E94702868
:103032000E94752812F40E94BF22E1E0E515E9F42E
:10304200062C0728D1F40E9470270E947E28A8F43B
:103052000E9482280E94702732960E94872868F474
:103062000E9450280E94B32C40F40E948B28E43620
:10307200A0E0FA0710F40E949028E1E0E51551F56E
:103082000E94352339F50E9482280E9470283097C9
:1030920011F40E9499280E94A02854F40E94462804
:1030A200159734F40E944B280E9450280E945528FC
:1030B2000E946B283CF40E9470280E94752812F42A
:1030C2000E94BF220E94A428A536E0E0BE0714F0A9
:1030D2000E94A9280E943A2311F40E94BF220E9452
:1030E200A428A436E0E0BE0714F00E94A928E1E07B
:1030F200E515D1F40E943F23B9F40E94E826119706
:1031020038F40E94ED260E94B02811F40E9437285C
:103112000E94ED260E94A428AE17BF072CF40E943D
:10312200322810F40E94B4280E94B7280E943C283A
:10313200E0932505F09326050E94BD28E13BA4E01B
:10314200FA0740F00E94B1220E94AA220E9402289D
:103152000E94C622E1E0E51581F5E3E0F0E06E169B
:103162007F0658F50E9470270E94872820F00E944F
:103172008B280E94EC250E948B28DF010E94B32C31
:10318200E0F40E947027DF010E94B32CB0F40E9489
:103192008B28E436A0E0FA0780F40E9490280E946F
:1031A2008B28EC59FF4FA0E3B0E00E94202B0E9435
:1031B2007827309711F40E94C228E1E0E51511F05A
:1031C2000C942D190E944628119714F00C942D1975
:1031D200F50131965F01E2E0F0E06E167F06E0F560
:1031E20000240A140B0420F4F501EC59FF4F5F018F
:1031F200E6E6F0E0EA15FB0590F00E9450280E94F6
:10320200B32C70F4E5E6F0E05F01EA15FB0541F44A
:103212000E9490280E94C828AC9A0E94C828AC98A4
:103222000E94B0270E94CE28EA15FB05A8F40E944E
:10323200BF220E94B8220E94AA220E94B1220E94AA
:1032420002280E94C62255240E94D3280E94D2221C
:103252000E94D2220E94E0220E94BD280E94EC25F8
:10326200E991EFBFF991E991B991A9919991899168
:1032720079916991F9901990099018951A930A9386
:10328200B89AC09A0E94D628C0980E94DE28E0937D
:103292003B05F0933C058BE18A95F1F70E94DE280D
:1032A200E0933F05F0934005C09AE0913B05F09111
:1032B2003C050E94E428DF01CB01E0913F05F0913B
:1032C20040050E94EC28AAE2B0E027C01A930A93B4
:1032D200A79AAF9A0E94D628AF980E94DE28E09360
:1032E2003D05F0933E058BE18A95F1F70E94DE28B9
:1032F200E0934105F0934205AF9AE0913D05F091CC
:103302003E050E94E428DF01CB01E0914105F091E6
:1033120042050E94EC28ACE2B0E00E94082B0E9419
:10332200FA28DF01CB01E0E0F0E068EC72E40E94F1
:103332006E2CADECBCEC8CEC9DE30E94D22BD80140
:10334200882799270E94F42A0E94202C0E94662B2B
:103352008F01F801099119910895E2E9F6E0FA93D3
:10336200EA930E943C280E9403270E94FF28EAE970
:10337200F6E0FA93EA930E94BD280E9403270E9476
:10338200FF28E2EAF6E00E9404290E94FF28EAEA06
:10339200F6E0FA93EA930E940B290E94FF28E2EBDF
:1033A200F6E00E941029E1E0E51521F4EAEBF6E0EF
:1033B2000E941029552021F4E1ECF6E00E94102928
:1033C200F301309719F4E8ECF6E01BC0E130A0E01D
:1033D200FA0719F4E4EDF6E014C0E230A0E0FA07CF
:1033E20019F4EDEDF6E00DC0E330A0E0FA0719F4B0
:1033F200EAEEF6E006C0E430A0E0FA0741F4E8EFB6
:10340200F6E0FA93EA9380E00E946D222296062C5F
:10341200072811F00C944E1AE42D0E94252319F46A
:103422000E9417293AC0E130A0E0FA0719F40E947D
:103432001A2933C0E230A0E0FA0719F40E941D29CC
:103442002CC0E330A0E0FA0729F4E8E2F7E00E949A
:10345200102923C0E430A0E0FA0729F4E6E3F7E0FC
:103462000E9410291AC0E530A0E0FA0729F4E4E42A
:10347200F7E00E94102911C0E630A0E0FA0729F413
:10348200E2E5F7E00E94102908C0E730A0E0FA0761
:1034920021F4E0E6F7E00E9410290E943523A1F40E
:1034A200ED2D0E94252319F40E9417290DC0E13049
:1034B200A0E0FA0719F40E941A2906C0E230A0E03F
:1034C200FA0711F40E941D290E943A23A1F4E82D63
:1034D2000E94252319F40E9417290DC0E130A0E0B3
:1034E200FA0719F40E941A2906C0E230A0E0FA078E
:1034F20011F40E941D290E943F2331F5EC2D0E94F8
:10350200252319F40E9417291FC0E130A0E0FA0711
:1035120019F40E941A2918C0E230A0E0FA0719F43F
:103522000E941D2911C0E330A0E0FA0729F4E8E265
:10353200F7E00E94102908C0E430A0E0FA0721F465
:10354200E6E3F7E00E9410290E94302321F4EEE620
:10355200F7E00E9410290895E0E8EBBBEABBE0E047
:10356200E8BBEFEFE7BBEFE6E5BBE0E9E4BBE0E099
:10357200E2BBE1BBE0E5E3B9E8E0E2B9E0E0E09319
:103582006200E0936100E0936500E0936400E0BFB5
:10359200E7E6E3BFE0E0E2BFE1BFEFBDE4E0EEBD9E
:1035A200E0E0EDBDECBDE7BDE6BDEAE7EBBDE2E183
:1035B200EABDE0E0E9BDE8BDE0937900E093780080
:1035C200EBE6E5BDE0E0E4BDE3BDE1E8E0938B00BE
:1035D200E5E0E0938A00E0E0E0938900E093880070
:1035E200E0938100E0938000E0938700E0938600FF
:1035F200E0938500E0938400E0938300E0938200EF
:10360200E0936A00EABFE0E5E9BFE8BFE0E1E7BFB7
:10361200E0E0E0937D00EBB9E8E1EAB9E6E0E093AF
:103622009500E0E0E0939000EFE2E9B9E0E8E8B964
:10363200E0E0E0BDE3E5EDB9E0E0EEB9E4E1EA9314
:103642000E943D20EFE1E1BDEFE0E1BD78940E94F0
:10365200CF1F0E940228662477240E949027E1E06F
:10366200E51511F00C94951C062C072811F00C940A
:10367200D81B0E948B27319741F40E9444270E9455
:1036820020290E94BD280E942D290E948B27309755
:1036920011F00C94981B0E9444270E9420290E943A
:1036A2003829319721F40E94BD280E942D290E94B9
:1036B20038293B9790F0AEE1B0E00E94082B0E94BF
:1036C2002D290E943D29EA0FFB1F0E944329AEE1EA
:1036D200B0E00E94082B0E94EC25E1E0E51539F5E7
:1036E2000E9497270E947E2810F50E943829319760
:1036F200A9F40E949C270E94E826EA0FFB1FE09390
:103702002305F09324050E9438293A96A4E0B0E0FC
:103712000E94202BAC9A0E944829AC980E945D26F8
:103722000E947E2820F40E94C2280E944E290E94F4
:103732003D29EA17FB0710F40E944E290E940A282D
:10374200B4F50E9450290E9455290E94632920F451
:103752000E946B29319603C00E946B293197FE9318
:10376200EE93A0911C05AA2312F40E9470290E94D4
:10377200772914F00E947F29A0913605AA2312F41A
:103782000E94B8220E9456273197A0913505B09128
:103792003605EA17FB0734F40E945627E0933505F5
:1037A200F09336050E94862910F00E948E290E940D
:1037B2003A2311F00C94211C0E9444270E942029D4
:1037C2000E94BD280E942D290E940A28CCF50E9441
:1037D20050290E9455290E943D29EA17FB0710F43F
:1037E2000E944E290E940A285CF50E9450290E94DC
:1037F20055290E94632920F40E946B29319603C047
:103802000E946B293197FE93EE93A0911C05AA2387
:1038120012F40E9470290E94772914F00E947F29D5
:10382200A0913605AA2312F40E94B8220E941E28F3
:1038320014F00E9426280E94862910F00E948E29E8
:103842000E943F2311F00C94951C0E94E8261297C7
:1038520010F40C94951C0E9444270E9420290E9477
:10386200BD280E942D290E940A28CCF50E945029C9
:103872000E9455290E943D29EA17FB0710F40E9475
:103882004E290E940A285CF50E9450290E9455295F
:103892000E94632920F40E946B29319603C00E9482
:1038A2006B293197FE93EE93A0911C05AA2312F483
:1038B2000E9470290E94772914F00E947F29A0910A
:1038C2003605AA2312F40E94B8220E941E2814F080
:1038D2000E9426280E94862910F00E948E290E94AA
:1038E2009129D001882799270E94B72CA8F40E9419
:1038F200BF220E94B8220E94AA220E94B1220E94E4
:1039020002280E94C62255240E94D3280E94D22255
:103912000E94D2220E94E0220E94BD28ED34A4E03F
:10392200FA0710F00E940228E1E0E51511F00C946C
:10393200961D062C072889F4A0913205AA236AF461
:103942000E94972914F40E949D290E946B282CF44E
:103952000E94A72912F40E94BF220E94352389F4F3
:10396200A0913205AA236AF40E94972914F40E94B6
:103972009D290E946B282CF40E94A72912F40E9410
:10398200BF22062C072811F00C941A1D0E947027E2
:103992000E94872810F40E94BF220E9470270E9472
:1039A200872810F40C941A1D0E94A028BCF40E94CF
:1039B2009D260E94B1290E9470270E94C829EA0F01
:1039C200FB1F0E94D0270E94CD2920F40E945D2671
:1039D2000E94D0270E94D2290E94D7290E947028D3
:1039E200309711F40E9499280E94E52920F40E9440
:1039F200EA29319603C00E94EA293197FE93EE9399
:103A0200A0911A05AA2312F40E94EF290E94F62916
:103A120014F00E94FE29A0913405AA2312F40E94F8
:103A2200BF220E94A92631970E94B02814F40E9456
:103A3200052A0E943523B9F50E94A0287CF40E9431
:103A42009D260E94B1290E94CD2920F40E945D2664
:103A52000E94D0270E94D2290E94D7290E94702852
:103A6200309711F40E9499280E94E52920F40E94BF
:103A7200EA29319603C00E94EA293197FE93EE9318
:103A8200A0911A05AA2312F40E94EF290E94F62996
:103A920014F00E94FE290E94A92631970E94B028A4
:103AA20014F40E94052A0E943F23A1F50E94ED26EC
:103AB2000E94B02834F40E94ED26E0933305F0937F
:103AC20034050E949129D001882799270E94B72C9A
:103AD200C8F40E94BF220E94B8220E94AA220E9419
:103AE200B1220E9402280E94C6225524A0E2B0E020
:103AF2000E94CD220E94D3280E94D2220E94D2226A
:103B02000E94E0220E94BD28ED34A4E0FA0710F0E2
:103B12000E940228E3E0F0E06E167F0630F40E9475
:103B22005D26309711F40E94BF22E1E0E515F1F520
:103B32000E94302311F5999904C00E940B2A0E9419
:103B420029279A9907C00E940B2AED91FD9131977E
:103B5200FE93EE93989902C00E94142A9B9902C088
:103B62000E94142ACF9909C00E941B2AA3E3B5E040
:103B7200ED91FD913197FE93EE930E941E2814F071
:103B82000E9426280E94A428A436E0E0BE0714F072
:103B92000E94A928A0913605AA2312F40E94B822F5
:103BA200A0913405AA2312F40E94BF220E94492741
:103BB200F301309729F40E949526E6E7F7E023C047
:103BC200E130A0E0FA0729F40E949526E0E8F7E048
:103BD2001AC0E230A0E0FA0729F40E949526EAE82A
:103BE200F7E011C0E330A0E0FA0729F40E9495261D
:103BF200E4E9F7E008C0E430A0E0FA0741F40E94EB
:103C02009526EDE1F2E0FA93EA930E941B20062C3E
:103C1200072811F00C94641EE42D0E94252339F428
:103C22000E94212AEEE9F7E00E9406234CC0E1300F
:103C3200A0E0FA0739F40E94212AE9EAF7E00E949B
:103C4200062341C0E230A0E0FA0739F40E94212A9B
:103C5200E4EBF7E00E94062336C0E330A0E0FA0767
:103C620039F40E94212AEEEBF7E00E9406232BC0D2
:103C7200E430A0E0FA0739F40E94212AE8ECF7E0E8
:103C82000E94062320C0E530A0E0FA0739F40E9422
:103C9200212AE2EDF7E00E94062315C0E630A0E0FB
:103CA200FA0739F40E94212AECEDF7E00E9406237C
:103CB2000AC0E730A0E0FA0731F40E94212AE6EEBA
:103CC200F7E00E9406230E943523F1F4ED2D0E94B5
:103CD200252329F40E94212AEEE9F7E011C0E13000
:103CE200A0E0FA0729F40E94212AE9EAF7E008C0D5
:103CF200E230A0E0FA0741F40E94212AE4EBF7E067
:103D0200FA93EA930E941B200E943A23F1F4E82DD1
:103D12000E94252329F40E94212AEEE9F7E011C02E
:103D2200E130A0E0FA0729F40E94212AEBEAF7E049
:103D320008C0E230A0E0FA0741F40E94212AE4EB35
:103D4200F7E0FA93EA930E941B200E943F2381F539
:103D5200EC2D0E94252329F40E94212AEEE9F7E0A6
:103D620023C0E130A0E0FA0729F40E94212AEBEAFD
:103D7200F7E01AC0E230A0E0FA0729F40E94212AF3
:103D8200E4EBF7E011C0E330A0E0FA0729F40E9467
:103D9200212AEEEBF7E008C0E430A0E0FA0741F494
:103DA2000E94212AE8ECF7E0FA93EA930E941B2092
:103DB2000E9449270E94F726E0EFF7E00E940623BF
:103DC200E0913505F0913605E0932B05F0932C0533
:103DD2000E94B72853DA8F010E940F26E7E0F8E02D
:103DE2000E9404290E94BD280E9403270E940B29D9
:103DF2008CE00E94592260960E940A230E940F269C
:103E02000E940E200E94482961DAE0934505F09352
:103E120046055CDA9F010E94A12530DAE093430552
:103E2200F09344050E940F26EBE1F8E0FA93EA933F
:103E3200F9010E9403270E94F127F8010E9403273B
:103E42008CE00E94592260960E94FD260E940F2655
:103E52000E940E200E947028EE0FFF1FE1BFE0912A
:103E62003505F0913605EE0FFF1FE09386000E94A4
:103E7200E0273196E3BDE4E0F0E06E167F0690F4B1
:103E82009A9B07C00E941B2A0E943E263196FE93EF
:103E9200EE93999B07C00E941B2A0E943E263197EF
:103EA200FE93EE930E945028A233E1E0BE0770F029
:103EB2000E945028AC32E1E0BE0730F4ECE2F1E0BF
:103EC200E0932105F09322050E94AA220E94BD28B8
:103ED200339720F40E94B8220E94BF22552021F479
:103EE2009B9902C0CF9BFECF38DAB9CBFFCFFFE060
:103EF200FA95F1F70895A1B3AF70A1BB919A90988A
:103F0200F6DF929AF4DFA0B39298F1DF929AEFDF94
:103F12009298A7FDF5CF0895A07FAB2BA2BB929AF2
:103F22000E94781F92980E94781F08959198A1B3D9
:103F3200A76FA1BBB2B3BF70A881EEDFA881A29523
:103F4200EBDF919A0C948522929A0E94781FE0B33B
:103F520092980E94781FE07F08950E94781FF4DFF4
:103F6200AE2FF2DF9198E295EA2B08950E947C1F12
:103F72000E94272AE65BFA4FE081F0E0DF01E98147
:103F8200F0E0EA0FFB1FEA930E94971FE981E0939A
:103F92004E05E881E0934F05229608950E947C1F0A
:103FA200E2E0EA930E94971F0E947C1FECE0EA93F2
:103FB2000E94971F0E947C1FE1E0EA930E94971FD4
:103FC200E0E0E0934F05E0934E050895EF93FF93F1
:103FD200A8816894AA3061F0E894E0914E05EF5F01
:103FE200E0934E05E0915005A0914E05EA1760F46A
:103FF200E0914F05EF5FE0934F05E0E0EA93E09137
:104002004F05EA93B3DF2EF076DF909AA881AA9348
:104012008DDFFF91EF910C9485221A93A981BA81C9
:10402200ED91A983BA831E2FE03019F01A93CEDFE7
:10403200F5CF0EC01A93E981FA813196E983FA83AA
:104042003197E4911E2FE03019F01A93BFDFF3CFBE
:10405200188123960895AA27BB271197F1F708958F
:104062009198A1B3A76FA1BBB2B3BF70A8810E9400
:104072008D1F919A0C94852292989098E881E093F2
:1040820050050E94272AE058FF4FE0934C050E94FA
:10409200272AE054FF4FE0934D050E942A2A0E94EE
:1040A2002A2A0E942A2AD7DFE0E2EA93D9DFD3DF65
:1040B200EAE20E94302AE4E00E94302AE5E80E9407
:1040C200302AA1B3AF70A1BB919A0E94AE1FE53016
:1040D20019F0E0E00C9485220E947C1FE6E0EA934E
:1040E2000E94971F0E94CF1FE1E00C9485225D9BE6
:1040F200FECFE881ECB908C21A930A93AC81BD8164
:104102000E94E52A3097C1F0AA81BB810E94E52A6C
:104112008F01309749F00230E0E01E0760F0F801AD
:1041220031978F01ED93FC93AC81BD810E942927C9
:104132003197AE81A08303C0EE81EA93D8DF198163
:1041420008812796089526970E94BC2C10E0EA89E0
:10415200FB893196EA8BFB8B3197E4912E2FE0306D
:1041620011F40C945522E12F0E94252339F42532B3
:1041720011F411E002C00E94352A95C1E130A0E09D
:10418200FA07A9F4253219F40E94352A8BC112E0EC
:1041920040E000E02D3211F401E085C12B3211F430
:1041A2004BE281C1203211F440E27DC104C0E23011
:1041B200A0E0FA0761F450E013E0203339F40E94E2
:1041C200402AE0E8F0E0EA2B0E2F6DC106C0E33092
:1041D200A0E0FA0711F00C945422203310F02A3395
:1041E20008F015C0A52FB0E0EAE0F0E0EA02F00125
:1041F2005E2F652F7727A22FB0E0E0E3F0E00E9468
:10420200FD2AEA1BFB0BDB01EA0F5E2F4CC10E9469
:10421200432AE336A0E0FA0749F40E94462AE889D5
:10422200F989A481AA930E944C2A3CC1E337A0E0F9
:10423200FA0741F40E94462A0E94562A0E948722C7
:104242001E2F11C0E037A0E0FA07D9F40E94462AD7
:104252000E94562A0E9491221E2F0E94402AE8E0C4
:10426200F0E0EA2B0E2F0E94402AE2E0F0E0EA2B77
:104272000E2F0E94402AEFE7FFEFEA230E2F30E0D5
:104282004FC0E436A0E0FA0721F0E936A0E0FA07D1
:1042920039F40E94402AE4E0F0E0EA2B0E2F04C039
:1042A200E537A0E0FA0731F4ECE8F0E0EE83FF83B3
:1042B20015E016C0E835A0E0FA0739F40E94402A5A
:1042C200E8E0F0E0EA2B0E2F06C0E837A0E0FA079C
:1042D20011F00C945322E6E9F0E0EE83FF8314E040
:1042E2000E94402A0E94602AB9F00E94462A0E9437
:1042F200662AAB85AA233AF4EA85FB850E94A82A9E
:10430200EA87FB874DE2403011F01F5F04C00E9434
:10431200402A0E946E2A04C00E94462A0E94662AEF
:104322000E94732AE9F41517D8F40E94402AE0E8A3
:10433200F0E0EA23FB23309771F00E94402A0E94AA
:10434200602A39F00E94402A0E946E2A242F1150BE
:1043520001C020E301C020E20E94352A5150E3CF80
:10436200312F0E94402AE2E0F0E0EA23FB2330975B
:1043720001F13030E9F00E94402AE8E0F0E0EA235F
:10438200FB23309741F0EE81FF813196EE83FF836C
:104392003197E49105C0AE81BF81ED91AE83BF83B9
:1043A200EA930E944C2A503009F051503150E1CF2B
:1043B2006EC020E3EE81FF810E94E92AE887F98737
:1043C200EE81FF813296EE83FF83E885F985AA8527
:1043D200BB85AE17BF0750F02F5FA885B985EA8568
:1043E200FB85EA1BFB0BEA87FB87EFCF2A3380F0C2
:1043F2000E94402AE8E0F0E0EA23FB23309721F014
:104402000E94432A379603C00E94432AB7962E2F52
:104412000E94402AE0E1F0E0EA23FB23309761F5B5
:10442200213320F4A885B985119709F410C05317D8
:1044320018F00E94732A09F024C020E20E94402A48
:10444200E0E8F0E0EA23FB233097B1F020E3A02F6D
:10445200B0E0E0E1F0E0EA2B0E2F0E94402A0E9439
:10446200602A51F00E94402A0E946E2A4A930E94BA
:104472004C2A503009F051500E94352A503009F030
:1044820051503150A885B985129708F092CF0E94F9
:10449200732A41F0503031F05150E0E2EA930E9429
:1044A2004C2AF8CF10E053CE0E94C32C6496089594
:1044B200FF920E94772ADE0116960E94802AEA83E2
:1044C200FB83DE0114960E94802A0E94852AAA811B
:1044D200BB81E0E0EC930CC0FF920E94772AE0E0FF
:1044E200EA83EB83DE0114960E94802A0E94852AC9
:1044F200198108812496FF900895E881EFB9EEB101
:10450200F0E0E078E1F3EFB121960895A991B99135
:10451200EE27FF276D91662311F03196FBCF0895A8
:10452200AA27BB27E991F9910590002011F0119675
:10453200FBCFFD0108950A921A92FA926A937A9336
:104542008A939A93AA93BA93EA93FA93EFB7EA9368
:104552000895E0E0F0E0E0932105F093220508954C
:10456200E0E0F0E0E0932305F09324050895E0E015
:10457200F0E0E0933505F09336050895E0E0F0E0D1
:10458200E0933305F09334050895ACE1B0E0E0E048
:10459200F0E00E94202B0895E0E0F0E00E94202B42
:1045A2000895AC9AE4EFF1E0FA93EA930E94932A19
:1045B200AC98E4EFF1E0FA93EA930C94932AAC9A64
:1045C200E4EFF1E0FA93EA930E94932AAC980895FB
:1045D200E0E0EA93EA930E94B71FEEE4F1E0FA9377
:1045E200EA930E941B20E0E0EA93E3E0EA930E9450
:1045F200B71FEEE4F1E0FA93EA930E941B20E0E099
:10460200EA93E1E0EA930C94B71FFA93EA930C94CD
:104612001B20E0E0EA93E2E0EA930C94B71FA0E0EB
:10462200B0E00E940C2B0895E1500E94282BEF5F0E
:104632000895EEE1F0E0FA93EA930C94932AEF5F87
:104642000E94282BE1500895F0E0309708950E94CF
:10465200CF1FE4EFF1E0FA93EA930C94932AE4E09B
:10466200F0E0E615F7050895E1E0F0E0E615F7055C
:104672000895E2E0F0E0E615F7050895E3E0F0E0E2
:10468200E615F7050895E7E4F2E0BFCFA4E3B0E052
:104692000E94082BE0932305F0932405A2E3B0E0E7
:1046A2000E94082BE0932105F0932205A0E5B0E0DB
:1046B2000E94082BAEE2B0E00E94202BA6E5B0E0FB
:1046C2000E94082BA0E1B0E00E94202BACE5B0E0F4
:1046D2000E94082BAEE0B0E00E94202B08950E94B9
:1046E200082BA2E1B0E00E94202B0895A6E3B0E0DF
:1046F2000E94082BA8E0B0E00E94202B08950E949F
:10470200082BAAE0B0E00E94202B08950E94082BFB
:10471200ACE0B0E00E94202B0895A5E1B1E00E9438
:10472200082BE0933905F0933A05A5E0B1E008952E
:104732000E94082BE0933705F09338050895ECE5C5
:10474200F2E063CFAEE3B0E00E94082BE0932305D2
:10475200F0932405ACE3B0E00E94082BE09321051E
:10476200F0932205A2E5B0E00E94082BAEE2B0E091
:104772000E94202BA8E5B0E00E94082BA0E1B0E047
:104782000E94202BAEE5B0E00E94082BAEE0B0E024
:104792000E94202B0895A0E4B0E00E94082BA8E01C
:1047A200B0E00E94202B0895A7E1B1E00E94082BFF
:1047B200E0933905F0933A05A7E0B1E00895E1E707
:1047C200F2E023CFA8E4B0E00E94082BE093230597
:1047D200F0932405A6E4B0E00E94082BE0932105A3
:1047E200F0932205A4E5B0E00E94082BAEE2B0E00F
:1047F2000E94202BAAE5B0E00E94082BA0E1B0E0C5
:104802000E94202BA0E6B0E00E94082BAEE0B0E0B0
:104812000E94202B0895AAE4B0E00E94082BA8E091
:10482200B0E00E94202B0895A9E1B1E00E94082B7C
:10483200E0933905F0933A05A9E0B1E00895AAE6BC
:10484200B0E00E94082BE0932305F0932405A8E62C
:10485200B0E00E94082BE0932105F0932205ACE61C
:10486200B0E00E94082BAEE2B0E00E94202BAEE640
:10487200B0E00E94082BA0E1B0E00E94202BA0E74C
:10488200B0E00E94082BAEE0B0E00E94202B089519
:10489200A4E7B0E00E94082BA8E0B0E00E94202B21
:1048A2000895ABE1B1E00E94082BE0933905F09343
:1048B2003A05ABE0B1E00895ACE7B0E00E94082B06
:1048C200E0932305F0932405AAE7B0E00E94082BA9
:1048D200E0932105F0932205AEE7B0E00E94082B99
:1048E200AEE2B0E00E94202BA0E8B0E00E94082BCC
:1048F200A0E1B0E00E94202BA2E8B0E00E94082BC9
:10490200AEE0B0E00E94202B0895A6E8B0E00E943D
:10491200082BA8E0B0E00E94202B0895ADE1B1E0A1
:104922000E94082BE0933905F0933A05ADE0B1E01F
:104932000895AEE8B0E00E94082BE0932305F093BF
:104942002405ACE8B0E00E94082BE0932105F09327
:104952002205A0E9B0E00E94082BAEE2B0E00E947E
:10496200202BA2E9B0E00E94082BA0E1B0E00E9457
:10497200202BA4E9B0E00E94082BAEE0B0E00E9438
:10498200202B0895A8E9B0E00E94082BA8E0B0E02F
:104992000E94202B0895AFE1B1E00E94082BE09322
:1049A2003905F0933A05AFE0B1E00895A0EAB0E02E
:1049B2000E94082BE0932305F0932405AEE9B0E0B2
:1049C2000E94082BE0932105F0932205A2EAB0E0B1
:1049D2000E94082BAEE2B0E00E94202BA4EAB0E0D5
:1049E2000E94082BA0E1B0E00E94202BA6EAB0E0D2
:1049F2000E94082BAEE0B0E00E94202B0895AAEAA4
:104A0200B0E00E94082BA8E0B0E00E94202B08959D
:104A1200A1E2B1E00E94082BE0933905F0933A0538
:104A2200A1E1B1E00895A2EBB0E00E94082BE0936F
:104A32002305F0932405A0EBB0E00E94082BE0933D
:104A42002105F0932205A4EBB0E00E94082BAEE210
:104A5200B0E00E94202BA6EBB0E00E94082BA0E160
:104A6200B0E00E94202BA8EBB0E00E94082BAEE041
:104A7200B0E00E94202B0895ACEBB0E00E94082B1E
:104A8200A8E0B0E00E94202B0895A3E2B1E00E94CA
:104A9200082BE0933905F0933A05A3E1B1E00895BC
:104AA200E4EFF1E0FA93EA930E94932A0C94CF1F69
:104AB200A2ECB0E00E94082BE0932305F0932405BA
:104AC200A5ECB0E00E94082BAEE2B0E00E94202BE1
:104AD200A7ECB0E008950E94082BAEE0B0E00E947F
:104AE200202B08950E940C2BA2E1B0E0F0E00E947E
:104AF200202B0895A9ECB0E00E94082BE093230537
:104B0200F0932405ACECB0E00E94082BAEE2B0E0DA
:104B12000E94202BAEECB0E00895A0EDB0E00E9420
:104B2200082BE0932305F0932405A3EDB0E00E9447
:104B3200082BAEE2B0E00E94202BA5EDB0E0089574
:104B4200E8ECF0E0FA93EA930C94932AA7EDB0E034
:104B52000E94082BE0932105F0932205A9EDB0E015
:104B620008950E94082BA0E1B0E00E94202B089536
:104B72000E94082BE0932105F09322050895A5EEEB
:104B8200B0E00E94082BE0932305F0932405A7EEE2
:104B9200B0E0A1CF0E94082BA3EEB0E00E94202B30
:104BA20008950E94082BE0932305F09324050895AD
:104BB200EEE2F3E02ACDE9E4F5E0FA93EA930C940D
:104BC2000E20A6E0B0E00E94082B089531970E94C3
:104BD200202B3196089531960E94202B319708950B
:104BE200659785E1A0E0B0E00895FE01FA93EA93AB
:104BF2000E940E2065960895A1E0B0E00E940C2B61
:104C02000895A2E0B0E00E940C2B0895A3E0B0E06A
:104C12000E940C2B0895EEE4F1E0F7CCE0E0F5E021
:104C2200FA93EA930895E3E4F3E0FA93EA93E091C6
:104C32002105F0912205662777270E94ED2A84E05C
:104C42000E9459222896E2E0EA93E3E0EA930E9466
:104C5200B71FE4CF0E940E20E0E0EA93E1E0EA937E
:104C62000E94B71FE2E5F3E0D0CCE0E0EA93EA93DA
:104C72000E94B71FE7E6F3E0C8CCA1E2B5E0ED91F0
:104C8200FD9108953197FE93EE93E2E3F0E0FA93FB
:104C9200EA930C94932A3196FE93EE93E2E3F0E0CA
:104CA200FA93EA930C94932AA0912105B0912205DC
:104CB200AD32E1E0BE070895E0912105F0912205B1
:104CC2000895E3E4F3E0FA93EA930895A3E0B1E0F0
:104CD2000E94082B0895662777270E94ED2A84E018
:104CE2000E9459222896E2E0EA93E3E0EA930E94C6
:104CF200B71F94CFE2E3F0E0FA93EA930C94932A7D
:104D0200ECE7F3E0FA93EA93A0E1B0E00E94082B0B
:104D1200E2CF0E940E20E0E0EA93E1E0EA930E94F3
:104D2200B71FE0E9F3E071CCE0E0EA93EA930C9478
:104D3200B71FE5EAF3E069CCA0E1B0E00E94082BDE
:104D42000895A0E1B0E0EFE0F0E00E94202B08958A
:104D5200E0913705F091380508950E94C02A0E941B
:104D6200ED2A84E00E9459222896E2E0EA93E3E0E9
:104D7200EA930E94B71F52CFED91FD9183CFED913F
:104D8200FD9189CFE4E6F0E0E0933705F093380532
:104D92000895E0912305F091240508950E940E20C4
:104DA200E0E0EA93E1E0EA930E94B71FEAEDF3E064
:104DB2002CCCA3E2B5E0E0CFA3E2B5E0E0CFA09136
:104DC2002305B0912405AB3EE1E0BE070895A09112
:104DD2002305B09124050895A3EEB0E00E94082BAC
:104DE2000895E4E6F0E00E94202B0895E0E0EA93C3
:104DF200E1E0EA930C94B71FE0E0EA93E3E0EA9380
:104E02000C94B71F662777270E94ED2A089588E041
:104E12000E9459222C960895A6E1B0E00E94042B2C
:104E22000895ED91FD913197FE93EE93F5CFE13028
:104E3200A0E0FA07A0E06A07A0E07A070895A6E1D9
:104E4200B0E0E0E0F0E060E070E00E94182B08952E
:104E5200ED91FD913196FE93EE930895A6E1B0E0B7
:104E62000E94182BADE1B5E00895E0931D05F09383
:104E72001E050895ECE7F3E0FA93EA93AEE0B0E0A2
:104E82000E94082B28CFAEE0B0E00E94082B0895C4
:104E9200E4E6F0E0FA93EA930C94932AAEE0B0E0F1
:104EA200EFE0F0E00E94202B0895E0913905F091A7
:104EB2003A050895E4E6F0E0E0933905F0933A0507
:104EC2000895E7E7F4E0FA93EA93AEE2B0E00E94D5
:104ED200082B98CF84E00E94592228968DCFAEE20B
:104EE200B0E00E94082B0895EAEDF3E08ECBA2E138
:104EF200B0E00E94082B0895A2E1B0E04DCBE6ECB1
:104F0200F4E083CBEBEDF4E080CBA2E1B0E00E94D1
:104F12000C2B0895A8E0B0E00E94082B0895A4E0AD
:104F2200B0E0E1E0F0E00E94202B0895AAE0B0E0BA
:104F32000E94082B0895ACE0B0E00E94082B08956F
:104F4200AAE2B0E00E94082B089584E00E94592250
:104F520028965FCBACE2B0E00E94082B0895A4E152
:104F6200B0E00E94082B0895E2ECF1E00E94202BB1
:104F72000895E1E0F0E00E94202B0895E6E1F0E0E0
:104F82000E94202B0895EFE0F0E00E94202B08956C
:104F9200E0E0F0E0E0931105F09312050895E0934C
:104FA2001705F09318050895E0E0F0E0E093190585
:104FB200F0931A05E0931B05F0931C050895A7E2F0
:104FC200B1E00E94082B0895E3E2F6E01ECBE8E38D
:104FD200F6E01BCBECE4F6E0FA93EA93DADE12CFCA
:104FE2006BDE10CF0E940E20E1E05E2EAA24BB24CD
:104FF200CCCAE6E5F6E0FA93EA93F2CFA0E3B0E09A
:10500200CBCAAAE1B0E0C8CAA0914505B091460555
:105012000895A0912D05B0912E050E94B32C0895FC
:10502200E0913505F09136053F97E0933505F09311
:105032003605A0913605AA230895A0913505B091B1
:105042003605A436E0E0BE070895E4E6F0E0E0931A
:105052003505F09336050895E0914505F091460532
:10506200089597DED1DFAE17BF070895A0E2B0E042
:105072000E94082BB0CDE0914305F09144050895BC
:10508200A0914305B09144050895A0913105B091D6
:1050920032050895E0914705F09148050895A091E1
:1050A2002105B09122050895AE0FBF1FEAE0F0E09E
:1050B2000E94CA2ADF01E3E2F0E00E94D22AE093D2
:1050C2003305F0933405E6DF3A96E0934705F09313
:1050D20048050895DADFAD3FEFEFBE070895E0918E
:1050E2003305F091340508957497E0933305F093F6
:1050F2003405A0913405AA230895C2DFEA17FB07FD
:105102000895ACE1B0E00E94082B65CDB9DFAE177F
:10511200BF070895A0E3B0E00E94082B0895AC9A5F
:10512200E0E9F1E0FA93EA930E94932AAC98089599
:10513200E3E2F0E0E0933305F09334050895A5DF50
:105142000E94B32C0895A0913305B09134050895BF
:10515200E4E6F0E0E0933305F09334050895F3DFDD
:10516200EA17FB070895A3E3B5E072CEB8DFE09338
:105172002905F0932A050895AAE1B0E00E94082BC0
:1051820008956ADFE0932305F09324050895E0E98A
:10519200F1E0FA93EA930C94932AA4E6B0E00E9419
:1051A200CA2A0895AA24BB2429CFE3E5EDB9E0E099
:1051B200EEB9B99ABA9ABB980895E0E0EA930E94D0
:1051C2007E22F0E0089566277727DF01CB01E8E031
:1051D2000E94B42A0895662777270E94A32A8F0186
:1051E200087F1F77169507951695079516950795CB
:1051F20008950E94C02A0E949F2B089584E00E9475
:105202006D2226960895FA93EA93E0912B05F09188
:105212002C05F8CDE0912905F0912A05F3CDFA93FA
:10522200EA9380E00E946D2222960895E3E0F7E07F
:10523200F6CFE1E1F7E0F3CFEAE1F7E0F0CFDF010B
:10524200EAE0F0E00E94D22AD4DFA3E1B5E00E94B6
:10525200662BED93FC930895A0911305B09114056C
:105262000E94CA2AE0931105F09312050895A4E062
:10527200B0E00E94082B08958CDDA0911105B09139
:1052820012050895E0931105F09312050895ECE2DA
:10529200F1E0FA93EA930C94932A7BDDF3CFE09149
:1052A2001105F091120579CFDF01E0911B05F09114
:1052B2001C05E650FF4F0E94D22AE0933505F09379
:1052C20036050895C9DEA0911105B0911205AE17F9
:1052D200BF070895ABE1B5E0ED91FD910895E0E0DF
:1052E200F0E0E0931B05F0931C050895A0911B05C7
:1052F200B0911C05AD32E1E0BE070895ECE2F1E0A9
:10530200E0931B05F0931C050895A0911105B0913F
:105312001205A33CE1E0BE070895E2ECF1E0B2CF52
:10532200A0E2B0E00E94082B0F0176CDAEDEEDEFD9
:10533200FFEFEA17FB070895B2DEE5E0F0E00E9416
:10534200D22AE0933305F09334050895C8DE7E97A0
:10535200E0933305F0933405A0913405AA23089510
:10536200DF01EAE0F0E00E94D22A43DFA5E1B5E0E6
:105372000E94662BED93FC93ACE1B0E00E94082BF7
:10538200A0911505B09116050E94CA2A08CEA091D7
:105392001705B091180508958FDCF9DFEA17FB07AE
:1053A2000895E0911705F0911805F7CEDF01E0911D
:1053B2001905F0911A05EA56FF4F0E94D22AE0938E
:1053C2003305F0933405089556DEE1DFAE17BF07CB
:1053D2000895A9E1B5E0ED91FD910895E0E0F0E0D6
:1053E200E0931905F0931A050895A0911905B0915B
:1053F2001A05AD32E1E0BE070895ECE2F1E0E09378
:105402001905F0931A050895A3DCE0933305F09390
:1054120034050895E9E1F0E0FA93EA930E94932AB1
:10542200A5E3B5E00895E9E1F0E0FA93EA930E947A
:10543200932A99CEE9E1F0E0FA93EA930C94932A45
:10544200EAE0EA93E0E0EA930C94B71FE881F0E027
:1054520008950E942C20E0E3EA930C943120EA9311
:105462000E94971F0C942C202A93EF85F889FA93B7
:10547200EA93FE013F96FA93EA930C947D20A02FC3
:10548200B0E00895E22FF0E00895E889F9893497B1
:10549200E88BF98B0895EF85F889FA93EA93FE0178
:1054A2003F96FA93EA930C947D20A889B9891496C1
:1054B2000E94E52AEE83FF83FA93EA930895E4E0DB
:1054C200F0E0EA23FB2330970895A889B98914965E
:1054D2000E94E52AEA87FB870895EBEFFFEFEA23B4
:1054E2000E2F0895E02FF0E0E1700895F82E229734
:1054F2001A930A93DE010E949F2A8D0108950E9449
:105502009F2A0E94E52A0895FA93EA931A930A932E
:10551200FE013696FA93EA93E0E0F0E0FA93EA931A
:105522000C94A420E991F991309639F080ED97E03E
:105532000197F1F7A8953197C9F708950024AF0DA7
:10554200B01D0895EA2BFB2B682B792B0895F1955A
:10555200E195F0400895F09560957095E195FF4FC3
:105562006F4F7F4F0895EE230E2EFD01BC0131F0E7
:10557200EE0FFF1F661F771F0A94D1F708956F2F52
:10558200660F660B762F08958B2F880F880B982F46
:105592000895FA9FF02DEB9FF00DEA9FE02DF10D9B
:1055A20008950024112490E1AA0FBB1F001C111CB6
:1055B2000E1A1F0A18F40E0E1F1E01C0A1609A9542
:1055C20099F7FD01D0010895ED91FC91119708958D
:1055D2000590F491E02D08957A936A93FA93EA93F1
:1055E2000895689401C0E89401D0A9D0182E862F9E
:1055F200612D192E972F712D1B2EBF2FF12D1A2ED3
:10560200AE2FE12D0895129602D0BF011297119686
:1056120002D0FE2F1197E199FECFFF93FFB7F894C6
:10562200AEBBBFBBE09AEDB3FFBFFF91089507D0B9
:1056320012960F01FB0103D0F0011297089507D0D3
:105642001196EF93EF2F03D0EF9111970895E19BFD
:1056520002C0A895FCCF9FB7F894AEBBBFBBE09A3F
:105662008DB3E81719F0EDBBE29AE19A9FBF089556
:10567200552342F4503811F4E0FF04C03196691FFB
:10568200791F6BF050E8572711F45F93C6C05F3F54
:1056920031F0660F000C57956795752F08955F934B
:1056A20000200AF0C6C0BFC050E8192E1522880F8C
:1056B200991F9527550F879550E8072E0522660FEB
:1056C200771F7527550F67950895689401C0E89470
:1056D2005F93F2DF703818F07F3F08F49EC056E106
:1056E200571BAAF4519558300EF4593030F0EFEFB1
:1056F200FFEF6FEF7FE777F91AC077275523B9F0ED
:10570200EE0FFF1F661F771F5A95D1F710C077273C
:10571200583028F0EF2FF62F672F5850F9CF552326
:1057220031F076956795F795E7955A95D1F7002070
:105732000AF411DF5F910895689401C0E8943097EC
:1057420060407040B1F0002426F0772312F40094F8
:1057520002DF172E7EE1112032F07A95EE0FFF1F45
:10576200661F111CF9CFEF2FF62F612D5F938ADF91
:105772005F9108954F93AF01FD01DA01AB01BC01C6
:10578200CA01402D012C142E4F910895EA0FFB1FE0
:10579200681F0895E095F0956095EF5FFF4F6F4F9A
:1057A20008955F9381DF903839F1703821F1572FD6
:1057B200591B13F112F4DEDFFACF583118F0AA2781
:1057C200BB278827583028F0AB2FB82F882758508E
:1057D200F9CF552329F08695B795A7955A95D9F70C
:1057E200502D512562F0D2DF38F46795F795E79591
:1057F200739513F41EC0BEDF45DF5F910895EA1B67
:10580200FB0B680B51F010F40094C4DF6623A2F383
:10581200EE0FFF1F661F7A95CBF7EE27FF2766274D
:1058220077275F910895EFEFFFEF6FE77FEF5F91CB
:105832000895EFEFFFEF6FE77FE75F9108955F93C2
:1058420033DF703851F3903841F301240894791F03
:1058520023F41CF300203AF3ECCF0F921F932F9303
:105862003F934F93112722279927689FA0018F9F6B
:10587200302D410D591F6B9F300D411D591F8E9FB9
:1058820027D0BF9F25D06A9F23D0BE9F1DD0AF9F38
:105892001BD0AE9F110D291F391F491F591FE32F1E
:1058A200F42F652F522F4F913F912F911F910F90FF
:1058B20066232AF0550FEE1FFF1F661F02C0739565
:1058C2004BF2D6DE5F910895100D211D391F02C0E3
:1058D200200D311D491F591F08955F93E5DE703871
:1058E20021F411200AF49FCFA4CF903809F495CF68
:1058F20001240894970B1BF4D4F30020F3CF792FE3
:105902001F932F933F934F9311241127222733275D
:105912004427552790E2AE17BF078607410730F0AC
:10592200AE1BBF0B860B410B089401C08894551F18
:10593200221F331F111CAA1FBB1F881F441F9A95C9
:1059420051F7F901612D4F913F912F911F916623DC
:1059520032F0550FEE1FFF1F661F7A9543F288DE65
:105962005F91089500240A160B060895EA17FB07B3
:105972006807790708955A934A933A932A931A9398
:105982000A9308955D814C813B812A8119810881A6
:105992000895AC0FBD1F05900D928A95E1F7089509
:00000001FF
